:030000000203B543
:0C03B500787FE4F6D8FD75813B0203FC64
:05000500012F01C10004
:02000B00610191
:10030100C0E0C0D075D008E5B0C4540FFFEF54036E
:10031100F521E5392521F522E52264026011E52266
:100321006404600BE522640B6005E522B40D20AF87
:100331002BAE2AAD29AC287BFF7AFF79FF78FFEF3E
:100341002BF52BEE3AF52AED39F529EC38F528E5B0
:100351002264016011E5226407600BE522640860F4
:1003610005E522B40E20AF2BAE2AAD29AC287B01C6
:100371007A0079007800EF2BF52BEE3AF52AED396A
:10038100F529EC38F528E52125E025E0F53920B6F9
:1003910010AF33AE32AD31AC308F2B8E2A8D298C1C
:1003A10028152FAF2FEF7007752F64D2A8D200D078
:0403B100D0D0E03296
:02000300814139
:10044100C0E0C0D0C2A8C200A20192B3752F6475EA
:100451003400E534D39527502A20B205E52FB401A5
:10046100F8E53B253BF53BE53A353AF53AA2D7921B
:100471000130B205E52FB401F8A20192B3C289059A
:080481003480CFD0D0D0E0326E
:10000D0075A800758922758C00D28CD288D2B975ED
:10001D00A883752F01E5B0C4540FFFEF5403FFEF14
:10002D0025E025E0F539E5B064FFFFEF5403F52C2D
:10003D00C3740A952CF527E52C700E75268475254D
:10004D0003752400752300801FE52CB4010E752661
:10005D00C2752501752400752300800C7526B475B5
:10006D002500752400752300AFA07E00EF7F00FEF4
:10007D00AD907C00EF2DFFEE3CFEEE64FFFEEF64D5
:10008D00FFFFE4FCFD7B107A007900780031CE8F04
:10009D00388E378D368C35AF38AE37AD36AC35EC56
:1000AD004D4E4F701A7F047E007D007C00AB26AA5A
:1000BD0025A924A82331CE8F388E378D368C357BEC
:1000CD00047A0079007800AF38AE37AD36AC359193
:1000DD00898F338E328D318C307B027A00790078A6
:1000ED0000AF38AE37AD36AC3591898F2B8E2A8D5A
:1000FD00298C283000FDC200E53824FFFFE5373498
:10010D00FFFEE53634FFFDE53534FFFCAB2BAA2AA7
:10011D00A929A828D3511D400C752B00752A0075EF
:10012D0029007528007F007E007D007C00AB2BAA86
:10013D002AA929A828C3511D5018E53824FFF52BED
:10014D00E53734FFF52AE53634FFF529E53534FF7B
:10015D00F5287B047A0079007800AF38AE37AD36DC
:10016D00AC359189C004C005C006C007AF26AE25C9
:10017D00AD24AC23AB2BAA2AA929A82831CED003B4
:10018D00D002D001D00091898E2D8F2EE52D64FFE8
:10019D00FEE52E64FFFFEF7805C333CE33CED8F9DD
:1001AD00F53B8E3AAF2CE53BAE3AA807088005C368
:1001BD0033CE33CED8F9F53B8E3AA2D7920121003A
:0101CD00220F
:1003C10002000DE493A3F8E493A34003F68001F245
:1003D10008DFF48029E493A3F85407240CC8C3333D
:1003E100C4540F4420C8834004F456800146F6DF0C
:1003F100E4800B0102040810204080900005E47E97
:10040100019360BCA3FF543F30E509541FFEE49300
:10041100A360010ECF54C025E060A840B8E493A3C7
:10042100FAE493A3F8E493A3C8C582C8CAC583CAF2
:10043100F0A3C8C582C8CAC583CADFE9DEE780BEAA
:01000A0000F5
:1001CE00E88FF0A4CC8BF0A42CFCE98EF0A42CFCD0
:1001DE008AF0EDA42CFCEA8EF0A4CDA8F08BF0A44E
:1001EE002DCC3825F0FDE98FF0A42CCD35F0FCEBAD
:1001FE008EF0A4FEA9F0EB8FF0A4CFC5F02ECD3972
:0F020E00FEE43CFCEAA42DCE35F0FDE43CFC22DE
:10048900C2D5E830E70FB2D5E4C39BFBE49AFAE49E
:1004990099F9E498F8EC30E717B2D51204BF1202C3
:1004A9006FE4C39BFBE49AFAE499F9E498F88003B2
:1004B90012026F30D50DE4C39FFFE49EFEE49DFD5B
:0404C900E49CFC2291
:10021D00EB9FF5F0EA9E42F0E99D42F0EC6480C858
:06022D0064809845F022F8
:1002330075F008758200EF2FFFEE33FECD33CDCC82
:1002430033CCC58233C5829BED9AEC99E582984005
:100253000CF582EE9BFEED9AFDEC99FC0FD5F0D6E2
:10026300E4CEFBE4CDFAE4CCF9A88222B800C1B90C
:100273000059BA002DEC8BF084CFCECDFCE5F0CB4A
:10028300F97818EF2FFFEE33FEED33FDEC33FCEB83
:1002930033FB10D703994004EB99FB0FD8E5E4F93E
:1002A300FA227818EF2FFFEE33FEED33FDEC33FC2B
:1002B300C933C910D7059BE99A4007EC9BFCE99A1F
:1002C300F90FD8E0E4C9FAE4CCFB2275F010EF2F64
:1002D300FFEE33FEED33FDCC33CCC833C810D70764
:1002E3009BEC9AE899400AED9BFDEC9AFCE899F89F
:0E02F3000FD5F0DAE4CDFBE4CCFAE4C8F92232
:00000001FF
